:030000000219FDE5
:03000B000200AA46
:03002B0002015D72
:03005B000202F1AD
:030073000202DEA8
:1000800002030406080C10182030406080040608A3
:100090000C10182030406080A0C00003070F1F0D17
:1000A0000D04050D050305030302C2AFC0D0C0E077
:1000B000206214E5256009E473E525F4F58AD2622F
:1000C000D0E0D0D0D2AF3285268AC262E526F46075
:1000D0003030682620720DD0E0D0D0C290C291C2DC
:1000E00092D2AF32C290C291C292206F0D20650AA7
:1000F0007401D5E0FDE57BF45290D0E0D0D0D2AFD2
:1001000032758A00C28DD26201FA01B930680520C9
:100110006502D29001B9306805206502D29101B91B
:10012000306805206502D29201B9D29330680A2066
:1001300065077405D5E0FDD29001B9D29430680A04
:100140002065077405D5E0FDD29101B9D2953068DC
:100150000A2065077405D5E0FDD29201B9C2AFC28D
:10016000AD53E6EFC0D0C0E0D2D3D2AFC2CEE52AC5
:100170006007207449152A21BE7800790020742E6A
:10018000E580307E01F430E70278FF53DACF207E3D
:100190000343DA20307E0343DA10C2D8C271E5800F
:1001A000307E01F430E70279FFC3E89970CB30610B
:1001B00003752A18207403752A18885CD27020747D
:1001C0000DE52B6004152B21CE43DA01C2D8207037
:1001D00002413DA85C206102C2702074367982B76A
:1001E0000431C3E894F0400374F0F8E8C4540F28D5
:1001F000F87984B703024113C313C313872120087E
:1002000002C313200A06C3C898F8411328F8500304
:1002100074FFF88822E52D54066022206B1FE53616
:10022000C333C333F8E564C313C313F9C395224042
:10023000028922E82522F52250037522FF7882B632
:100240000459852224A824C3E52495614002A861AD
:10025000C3E895634002A8638825E5667002418E75
:10026000C3E8AA669A5003E8FAE4F9EAC333FBE567
:1002700068F45B29400D2567F8E567600215674063
:100280000B418E0AC3E5679A5002056778FF8826FE
:10029000C26FC3E52694F84002D26F20CF0AD0E0A7
:1002A000D0D043E610D2AD32C2CF053A7801E52A6C
:1002B0006005307402152AC3E55C94014005755F42
:1002C0000041D4756000756900E55F2401F55F5059
:1002D00003755FFFD0E0D0D043E610D2AD32C2AF9D
:1002E00053E67F7592FA7593FFC260759104D2AFA1
:1002F00032C2AF53E6EFC2ADC0D0C0E0C0F0D2D33F
:10030000D2AFA8FBA9FCC2D8307102615853DACF32
:10031000207E0343DA10307E0343DA20D271E58079
:10032000307E01F420E702612F88278928A18553B8
:10033000DACF207E0343DA20307E0343DA10C2D8BE
:10034000C271307402A1717800E580307E01F43012
:10035000E702A171885CA15953DACF207E0343DA0A
:1003600020307E0343DA10C271206102813153DAFA
:10037000CF207E0343DA10307E0343DA20C2D8D286
:100380007188578958C3E89555F8E99556F97B0067
:100390007E087A00C3E8948CE994005005755B00F0
:1003A0008123882178A2E6A8216055C3E894C8E992
:1003B00094005008E4D2E4FB7A0A61FEC3E8946832
:1003C000E994015008E4D2E3FB7A0F61FEC3E8949C
:1003D000D0E994025008E4D2E2FB7A1E61FEC3E841
:1003E00094A0E994055008E4D2E1FB7A3C61FEC395
:1003F000E89498E994085008E4D2E0FB7A787E000B
:10040000C3E89559FCE9955AFD30E70AECF424015C
:10041000FCEDF43400FD755B00C3EC9AED9E5003D7
:10042000755B018859895A8557558558567802A1B8
:1004300059C3E89527F8E99528F9307C02A13D30A9
:100440007B02A13D307A02A1362075028154E9FD7C
:10045000E8FC8173E9C313F9E813F8307902A13697
:10046000E9C313F9E813F8307802A136E9C313FDA4
:0F047000E813FC20612CC3EC941CED94024002B5
:10047F00818AED701EC3EC94C850180529E52970C8
:10048F00021529C3E529940A5002A171755C00D2A7
:10049F0070A171E529600215297888E6F9740020AA
:1004AF007F087896B90302789EE624FAFEE43400BA
:1004BF00FFC3EC9EFCED9FFD9208B90310A20850FC
:1004CF0007207609D27681DC307602C276A20850F8
:1004DF0016B9030DECF42401FCEDF43400FD020415
:1004EF00F678007900A13DB90315EC33FCED33FD2F
:1004FF00C3EC940AFCED9400FD50047C007D00C316
:10050F00EC94FFED9400400678FF7900A13DEC8557
:10051F0072F0A4C5F0A2F733F87900400302055931
:10052F0078FF7900020559E9C313F9E813F8307C15
:10053F000EE9600278FFC3E81338F8E43400F9C31A
:10054F00E894FFE99400400278FF885CD270206144
:10055F0002A171741FF4552F4BF52FC274EB70026B
:10056F00D274752A18307403752A0A306102A18576
:10057F0020740353DAFE207403752B06D0F0D0E0FD
:10058F00D0D0D2AD43E6103279010205B57903021E
:10059F0005B5790A0205B5791E0205B5796402051C
:1005AF00B579C80205B57817E4D5E0FDD8FAD9F6C4
:1005BF00227A147B780205DC7A107B8C0205DC7AB8
:1005CF000D7BB40205DC7A0B7BC80205DCE573D525
:1005DF00E001227902E4D294D5E0FDD291D5E0FD7D
:1005EF00C291D5E0FDC294D5E0FDE920E002D290A2
:1005FF0030E002D292E573D5E0FDE920E002C2902F
:10060F0030E002C2927496D5E0FDD9C9EAF8D5E080
:10061F00FDD8FBDBB8D29422C37C007D0075F000BF
:10062F0005F0EA33FAEB33FB50F6EB13FBEA13FA60
:10063F00C3E9FFE8FEE89AF8E99BF95004EFF9EEF9
:10064F00F8B3EC33FCED33FDD5F0DFEDF9ECF82228
:10065F00E889F08A20D2D4F8A9F07B0030F70B7B21
:10066F00FFF42401F8E9F43400F9E88520F0A4AD93
:10067F00F0F8E98520F0A4AFF0FEED2EF974003FFD
:10068F00FA7C04C3EA13FAE913F9E813F8DCF48BE4
:10069F00F030F70AE8F42401F8E9F43400F9E889B6
:1006AF00F0C2D4F8A9F0227882B60403020711C36E
:1006BF00E55C940140030206DB852224E4F544F552
:1006CF0045F546F547F548C26E0207117882E6FCFC
:1006DF00D26EE522F523783879C7AA40AB41C3EB38
:1006EF0013FBEA13FAEC146013C3EB13FBEA13FAD0
:1006FF00EC14146007C3EB13FBEA13FAD1278844F9
:10070F00894522C3E5449523F8E5459400F9500C3B
:10071F00C3E89480E994FF4016020742C3E8947F30
:10072F00E994005003020742787F7900020742786C
:10073F008079FF8849894A22E5492546F8E54A35F7
:10074F0047F9854A20E4300701F43548FA30E709C4
:10075F00C3EA94F04015020780C3EA940F500302D6
:10076F00078078FF79FF7A0F020780780079007A87
:10077F00F0C3E5249561500AC374019524500B0210
:10078F00079EE54A20E70E02079EE54A30E70688F6
:10079F004689478A482278A5E6FAC3E54933F8E542
:1007AF004A33F9D15FE930E70BC3E89480E994FF4E
:1007BF004013E1D8C3E8947FE994005002E1D87860
:1007CF007F7900E1D8788079FFE820E715C3E5232A
:1007DF0098F84009C3E8940140030207FF7801022B
:1007EF0007FFE8F424012523F840030207FF78FFF1
:1007FF00884B2278A6E6FAA847A94812065FE93087
:10080F00E70CC3E89401E994FF4016020834C3E8EB
:10081F0094FFE99400500302083478FF790002082E
:10082F0034780179FFE920E715C3E54B98F84009C3
:10083F00C3E89401400302085B780102085BE8F407
:10084F002401254BF8400302085B78FF88242278A7
:10085F00FF20692879A1E76023E541601F74FF85B8
:0E086F0041F0848539F0306A0375F005A4F875
:10087D00C5F0600278FFC3E895645002A8648863F0
:10088D0022C3E5409440E5419401E5635003140112
:10089D009F046002F563220208A72275E890227872
:1008AD0083E6FF30EDF9A8BDA9BE0570C3E57094D0
:1008BD00084052757000E9FA79A0E76044EA7007C4
:1008CD00E571601B0208E0C3E895716010E5715099
:1008DD0006600C140208EC0460F90208ECE571F5F1
:1008ED0071C394F6401B7561C0C3940640137561C6
:1008FD0080C39406400B756140C394064003756137
:10090D000075BB0622E5612410500274FFF5617974
:10091D0082B704022139C3A861E524985002A824A6
:10092D00C3E895634002A86388258826E570B4075F
:10093D000375BB1022743279A787F0A4C5F0A2F716
:10094D0033F8C3E895614002A86188228824882580
:10095D0088268864227540007541F022C2AF75C8A3
:10096D0020A8CCA9CDAA3A30CF010A75C824D2AFA0
:10097D00AB3BAC3C883B893CC3E89BF8E99C2069C8
:10098D0008F9306602417821D2AD3D8A3DF9EA9DE4
:10099D00FA600478FF79FFAE3EAF3F8B3E8C3FA8E7
:1009AD003BA93CC3E89EF8E99FF9C3E54113FBE57C
:1009BD004013FAE82AF540E93BF54150067540FF32
:1009CD007541FF411FAA40AB41AC40AD417E047F54
:1009DD0002C3EB9404400D1E1FC3EB940840052089
:1009ED006A021E1FC3ED13FDEC13FCDEF7C3EA9C78
:1009FD00FAEB9DFBEF6009C3E913F9E813F8DFF794
:100A0D00EA28FAEB39FB8A408B4150067BFF8B407D
:100A1D008B41C3EB94025002D2663069047F0341CF
:100A2D004A7892E6FFC3E537948240110FC3E5374C
:100A3D0094A040010FC3EF940640027F057E02E5AE
:100A4D0041C4540FF9E541C454F0F8E540C4540FC6
:100A5D0028F8C3E89EFAE99400FB4009C3EA940222
:100A6D00EB940050047A02E4FB41C4AA40AB41EB85
:100A7D00C4FEEAC4540F4EFCC3EA9CFAEB9400FB8F
:100A8D00C3E813C313F8EA28FAEB3400FB8A408B52
:100A9D0041C3EB94024002C2667802EBC4FE7B00B8
:100AAD00EAC4540F4EFAC3EA98FA4005C3940250B3
:100ABD00027A027892E6FF30600241C48551928538
:100ACD005293D26043E680C3E49AF8E49BF9306612
:100ADD00026150E8FAE9FBD3E913FDE813FC8851F4
:100AED008952C3EF94036038EF20E00DE82CF8E94C
:100AFD003DF9ECFAEDFB020B19E828F8E939F9C3D9
:100B0D00E82402F8E93400F97AFE7BFFC3EF940381
:100B1D00400E8A538B54884D894E8C4F8D50618475
:100B2D00885389548A4D8B4E8C4F8D503069127578
:100B3D0053F07554FF754FF07550FF7551F07552A8
:100B4D00FF6184E8FAD3E813FC8851C3EF94036086
:100B5D0020EF20E007E82CF8ECFA6170E828240279
:100B6D00F87AFEC3EF940340088A53884D8C4F6189
:100B7D008488538A4D8C4FE568C3335002646BF5FE
:100B8D0068306002618E753402D26043E680E52DD7
:100B9D0054066034A840A941C3E913F9E813F8C31A
:100BAD00E913F9E813F8306904E92440F9C2AF53A9
:100BBD00E67F759100C3E498F594E499F5957591E8
:100BCD0004D26043E680D2AF22D264754300752013
:100BDD0000306C03752040020BF5D264754300752F
:100BED002040306C0375200078017901206620E5E6
:100BFD002D54066002C2647914E541C313700104DB
:100C0D00F8C3941440027814306904781B791B20C2
:100C1D006010E543600C306903D53404D26D81A0BA
:100C2D0071960543E59BF45440B52002818A3069E5
:100C3D000908C3E899400118811C20640A08C3E81B
:100C4D0099400261F5811CC264C2AF53E67F759174
:100C5D00003066127594007595F8759104D2604355
:0F0C6D00E680D2AF61F5E5417EFFC3334005C39A
:100C7C00334001FEC3E49E759400F5958167C3E58E
:100C8C00339401500261F530640261F5D802819E03
:100C9C00811CC26DC2AF53E67F759100855394855C
:100CAC005495759104854D92854E93D26043E680A0
:100CBC00D2AFE52D54066008206A020533020CDC25
:100CCC00306D0D206C0A2064071581158102158B7F
:100CDC002278003064027801E53775F007A4F9E555
:100CEC00F028F5F0E9A2F013A2F113A2F213F537F4
:100CFC00C394785003753778C3E53795384008D2DC
:100D0C0065C290C291C292306002A113854F928548
:100D1C005093D26043E68022207D16C2AF7542020A
:100D2C00D294C293306202D292D2AF759F11020F4D
:100D3C0013C2AF754202D294C295306202D290D2E5
:100D4C00AF759F11020F13307243207D20C2AF7517
:100D5C00420390013B757B10C292D295306204D253
:100D6C0091A171C294D2AF759F01020F13C2AF75DE
:100D7C00420390013B757B10C290D293306204D237
:100D8C0091A191C294D2AF759F21020F13207D17B0
:100D9C00C2AF754203900116C292306202D291D258
:100DAC00AF759F01020F13C2AF754203900116C2BB
:100DBC0090306202D291D2AF759F21020F13207D29
:100DCC0016C2AF754204D293C295306202D291D250
:100DDC00AF759F21020F13C2AF754204D295C29317
:100DEC00306202D291D2AF759F01020F1330724361
:100DFC00207D20C2AF75420590012A757B08C291F7
:100E0C00D294306204D290C117C293D2AF759F11A5
:100E1C00020F13C2AF75420590014C757B20C29135
:100E2C00D294306204D292C137C295D2AF759F1161
:100E3C00020F13207D17C2AF75420590010CC291B1
:100E4C00306202D290D2AF759F11020F13C2AF75F0
:100E5C004205900120C2913062EBD292D2AF759FC5
:100E6C0011020F13207D16C2AF754206D295C294A3
:100E7C00306202D290D2AF759F01020F13C2AF75D0
:100E8C004206D293C294306202D292D2AF759F21A5
:100E9C00020F13307243207D20C2AF7542019001C6
:100EAC004C757B20C290D293306204D292C1BDC2E9
:100EBC0095D2AF759F21020F13C2AF7542019001FD
:100ECC002A757B08C292D295306204D290C1DDC2E1
:100EDC0093D2AF759F01020F13207D17C2AF7542DD
:100EEC0001900120C290306202D292D2AF759F2144
:100EFC00020F13C2AF75420190010CC29230620214
:100F0C00D290D2AF759F01C2652290010A757B0009
:100F1C00C290C291C292D293D294D295C2622278DC
:100F2C008076090876090876040876FF08760308A7
:100F3C0076FF08760B087603087601087601788C24
:100F4C0076010876FF0876FF0876FF0876FF0876AC
:100F5C00FF0876030876FF0876FF0876FF087625EB
:100F6C000876D00876280876500876040876FF08AC
:100F7C00760208760008767A0876FF0876010876FD
:100F8C0001087600087603087600227887E6FFC20F
:100F9C0072BF0302D2727888E6C394036008C27DE4
:100FAC00E630E102D27DC27E7889E630E102D27E63
:100FBC00C3EF94026008758E01D273020FCF758E49
:100FCC0000C273227880E6149000809378A5F6789E
:100FDC0081E6149000809378A6F67886E61490004B
:100FEC008D9378A7F67886E6F539C394025003758D
:100FFC003902789CE67538FFB402037538A0B40347
:10100C000375388278A3E61490009A93F566120F54
:10101C001622227896E6FA7897E6FB7888E6B403EF
:10102C0005C3EB940EFB307F047A007BFFC3EB9A75
:10103C00FCC3948250027C827572000572EC85723E
:10104C00F0A4C3E5F0947D40F222D27F111F12056B
:10105C00A61205A67A007B007C1012059CE55C2A82
:0F106C00FA74003BFBDCF37C04C3EB13FBEA13C9
:10107B00FADCF7FEC27F111F22757C00757D00E53F
:10108B00EF20E6037520000520903FFFE52014605C
:10109B0006901DFF1460009304600375EF1453D981
:1010AB00BF7581C043FF8012059775EF0443B203F0
:1010BB00E5B3240220E70DF521E5E320E0068521C9
:1010CB00B343E301120F167580FF75A40075F19001
:1010DB0075D47F75903875A53F75F23F75D5007542
:1010EB00A60175E241120F16E4F8F6D8FD756801FA
:1010FB00120F2B1215DC78988673753001C2AF1264
:10110B0005B01205C01205A61205C71205A61205D9
:10111B00CE1205A6C2AF757C00757D0078FA79FA00
:10112B00308707D9FBD8F7021C00120F97120FD08C
:10113B00111E111F78988673120F167588107589FA
:10114B000275C82475910475D84075A82275B8022C
:10115B0075E690759B80759D0075D10775BC5875AC
:10116B00BB0675BA1175E880120597D2AF1208A4A9
:10117B0075360053DACF207E0343DA20307E0343EB
:10118B00DA1043DA01C2D8C2711205B0D2617B0307
:10119B007A0CE55B70077A0CDB0302111F1205A6B4
:1011AB0020700302111FC270E55CC3940240E1E59D
:1011BB002F541F855E5DF55EB55DD5DAD5C26153E3
:1011CB00DACF207E0343DA20307E0343DA10C2D815
:1011DB00C27178A2E67008D274E52F54E0F52FC2E5
:1011EB00757529001205AB307409C3E529940A40C3
:1011FB0002D27512059C78023074027800C3E55C4C
:10120B009840F0C2AF1205C01205C01205C0D2AF94
:10121B001205B0754C007888E6B403026114120510
:10122B009C788CE6C394015003021314E530C394ED
:10123B00015003021314757CA5757DF1207435C321
:10124B00E55C94FF5003021314C2AF1205D5D2AF65
:10125B001205ABC3E55C940150EFC2AF1205C0128F
:10126B0005A11205C0D2AF1205ABC3E55C94FF40DC
:10127B00E90217887F02D27F111F1205ABC2AFC2E2
:10128B007F111FAE5CC3E55C947FD2AF500261242B
:10129B00120597C2AF1205D5D2AFDFDA1156C3EEE6
:1012AB007897F61205B012170B7F0AD27F111F1217
:1012BB0005ABC2AFC27F111FAE5CC3E55C947FD29E
:1012CB00AF50E6120597C2AF1205C01205A1120569
:1012DB00C0D2AFDFD61156EE24037896F6F8799785
:1012EB00E7C394824003985006E824827897F6125D
:1012FB0005B012161E12173A1205AB111FC3E55C8F
:10130B0094FF50024141021788757C00757D00C324
:10131B00E55C954C4003855C4C1205AB78017988F4
:10132B00E7B403027805C3E55C9840024121C2AFE4
:10133B001205D51205D51205D5D2AF1205B07530F1
:10134B0000E4F531F5320531E531F4703F053278C3
:10135B009AE67819146012783214600D787D146057
:10136B000878FA146003753200C3E53298401D12F9
:10137B000F16120597153275310078998673C2AF27
:10138B001205D5D2AF789886731205AB1205A1E57D
:10139B002A7005307402211F78012074027806C36D
:1013AB00E55C9840A17888E6C3940360031205AB13
:1013BB00E52A700302111FC2AF120F16E4F522F5D6
:1013CB0023F524F525F526F567D2AF7885E6C333EB
:1013DB00F565E4F544F545F546F547F548F570F543
:1013EB002CF52DF53775700875BB10120597120883
:1013FB00A830EDFDA8BDA9BEE97001F888711208EF
:10140B00AC75700875BB10120F97C2AF7561FF12E8
:10141B000942852261852262852263D2AF75220142
:10142B00752401752501752601856069756A01783A
:10143B0088E6B40307C27D307602D27DD268D269CA
:10144B00753300120E70120E9F1209621209691287
:10145B000962120969120962120BE71206B6120C25
:0D146B00DD120D24120969120BD6306E033C
:1014780012071220660312085E30660312088E12E5
:101488000CDD120D53120969120BE7306E031207B7
:1014980047120CDD120DCA120969120BD6306E0301
:1014A8001207A5120CDD120DF9120969120BE730AB
:1014B8006E03120802120CDD120E7012096912086E
:1014C800A8120BD6120CDD120E9F1208AC12096975
:1014D800306932856461856462856069756A0179FD
:1014E800187A0CC3E53399400FC269D26A8A3585E8
:1014F800646185646302150DC3E55C9401400302D1
:101508001463021593306A1D206C1AE535147006B1
:10151800C26AD26B8163F535C3E55C94014003026E
:10152800146302159375360078FA79A4E760027897
:1015380003C3E55F985054307404E52A604D7888F9
:10154800E6B40317207D05207607A163307602A153
:1015580063206C07D26C85646181A278F0306C05D9
:101568008564617820C3E5419850028163306C1B23
:10157800C26CC27D307602D27DD26A75351285641E
:101588006181630536E55C6002A196753600C2AFDD
:10159800120F167887E6FE7602120F977887EEF616
:1015A800E4F522F523F524F525F526F565752C00D7
:1015B800752D00D2AF1205AB120F1678A4E660069F
:1015C800D290D291D292307409C3E5369404400285
:1015D800211F614C901A0D7820121660E520B45531
:1015E8000CA3121660E520B4AA030215FE120F2BF5
:1015F80012161E02161D901A0378807B0A121660B6
:10160800A308DBF9901A0F788C7B19121660A308CF
:10161800DBF9901A2822C2AF1216A3121680901A6C
:1016280000740E121665A37407121665A3741512BA
:101638001665901A0378807B0A121664A308DBF9F2
:10164800901A0F788C7B19121664A308DBF912160E
:10165800B6121694901A2822E493F622E6438F01D4
:10166800538FFDFFC3E583941C400122EF857CB7AF
:10167800857DB7F0538FFE22438F02438F01857C0F
:10168800B7857DB7901A0DF0538FFC22901A0D7410
:1016980055D165901A0E74AAD165227A3079D0781E
:1016A80020901A40D160E520F709A3DAF7227A30B2
:1016B80079D0901A40E7D16509A3DAF922AB74A86A
:1016C80075BB01027980BB02027981BB0302798272
:1016D800BB04027984BB05027986BB06027992BBFA
:1016E80007027987BB080279A3BB0902799CBB0A68
:1016F800027988BB0B027989E8F7227C051205B0CC
:10170800DCFB22C2AF1205C01205C71205CE1205B6
:10171800D51205A11205C01205C71205CE1205D5AE
:101728001205A11205C01205C71205CE1205D5D2A1
:10173800AF22C2AF1205D51205CE1205C71205C0D9
:101748001205A11205D51205CE1205C71205C01241
:1017580005A11205D51205CE1205C71205C0D2AFD4
:1017680022AE74AF75C2AF1205C01205C01205C013
:101778001205A1DEF21205D51205A1DFF8D2AF22BB
:10178800F10BF103F103757401757501757600F1BC
:10179800697C05AD5C1205B0C3ED955C70F5C3E5D9
:1017A8005C9401400AC3E55C94FF40320217C4D13F
:1017B800C5D11EF10BC2AF75EF14F103DCD5057668
:1017C800C3E5769403500280C6F1030575E57414E9
:1017D80090009F93F808C3E57598500280AEF10316
:1017E800F1030574C3E574940C5002809C120F2B0E
:0A17F800D11EC2AF75EF14121703E3
:0319FD0002108451
:101A00000E0715090904FF03FF0B03010155AA0185
:101A1000FFFFFFFFFF03FFFFFF25D0285004FF0259
:091A2000007AFF0101000300FF40
:101A40002345415A5933417632232020202020203B
:101A500023424C48454C4923463333302320202031
:101A60002020202020202020202020202020202076
:101C0000C2AFC2D353D9BF7581C043B20343FF8073
:101C1000752438752503B1DC7529A5752AF175E29F
:101C20004043F18053A47F75D4FFD2877DFA7803B7
:101C300079E67C10752200752300901DE97B0675FE
:101C400024987525013087028145208708D8FBD963
:101C5000F9DCF781B7308708D8FBD9F9DCF781B711
:101C6000B19CE493A3C39A6004DDC381B7DBDBB10D
:101C70008E6002812E7B08E493FAA3B16FDBF87AC1
:101C800030B16F752200752300B18EEAFCEBFDC305
:101C9000ED94FE400EB18E8A278B28ED30E0048A49
:101CA000828B83B18E7AC270D8C3ED94FE601950D6
:101CB000CEBD002BEC600F7520007521FF7529004B
:101CC000752A000200008100A827A9280809D80465
:101CD000D90281DCB192EA89AAF281CE0D81A3C337
:101CE000ED94035053EDA2E092007AC5C3E58294CF
:101CF00000E583941C508A200010438F02438F011B
:101D00008529B7852AB7F0300029A827A92808090E
:101D1000438F01538FFDD804D902A133C3E58394C7
:101D20001C4003A3A11689AAE28529B7852AB7F02A
:101D3000A3A116538FFC817F7AC1BD030CE493A34A
:101D4000FAB153DCF8B14B817F8181AA22AB23B178
:101D50006FEBFAEA6222752608C3E52313F523E543
:101D60002213F52250066323A0632201D526EAB18F
:101D7000DCB1DC75260AEAF4200102D287300102C8
:101D8000C287B1DCC3134002C201D526EB22B19257
:101D9000EAFB208702A192308702A197752608AE40
:101DA00024AF25C3EF13FFEE13FEB1E0B1DCC3EAAD
:101DB000133087024480FA30E703632201C3E5232E
:101DC00013F523E52213F52250066323A0632201B5
:101DD000D526D9E52265236523F52222AE24AF2539
:101DE0000E0FDEFEDFFCD20122424C48656C6934E6
:071DF000373163F3300601F7
:00000001FF
